:100000000C940D010C9445010C9445010C94450190
:100010000C9445010C9445010C9445010C94450148
:100020000C9445010C9445010C94C91E0C949B1F23
:100030000C94BD190C9445010C9445010C94450198
:100040000C9445010C9445010C9445010C94450118
:100050000C9445010C94451A0C9445010C944501EF
:100060000C9445010C9445010C9445010C944501F8
:100070000C9445010C9445010C9445010C944501E8
:100080000C9445010C9445010C9445010C944501D8
:100090000C9445010C9445010C9445010C944501C8
:1000A0000C9445010C9445010C9445018C038C0380
:1000B000B803B80320043E04560556054904E2047B
:1000C000F304F30408202F2027212F2027217B2051
:1000D0009E202721F52004212100220023001E005C
:1000E0001F00200028004A00A80014034900530004
:1000F0004F0020004D006100630072006F0000009F
:100100000C034D00650072006700650000000403E9
:10011000090409023B00020100A0FA0904000001E1
:10012000030101000921110100012240000705819E
:100130000308000109040100010300000009211166
:10014000010001227B00070582032000011201004B
:100150000200000008654D001201000102000105C7
:10016000010902A10185020901A10005091901295E
:10017000081500250195087501810205010930095E
:10018000311581257F95027508810609381581256D
:100190007F950175088106050C0A38021581257FB7
:1001A000950175088106C0C005010980A10185037C
:1001B00019012AB700150126B700950175108100B5
:1001C000C0050C0901A101850419012AA00215012D
:1001D00026A002950175108100C005010906A10144
:1001E000050719E029E71500250195087501810229
:1001F0009501750881010507190029FF150026FFE3
:1002000000950675088100050819012905950575F1
:10021000019102950175039101C011241FBECFEF1A
:10022000DAE0DEBFCDBF04B603FE18C080915102F4
:1002300090915202A0915302B09154028730904B9A
:10024000A740B04B59F410925102109252021092F2
:10025000530210925402E0E0F8E3099511E0A0E0A7
:10026000B1E0ECE4F4E402C005900D92A639B107C8
:10027000D9F722E0A6E9B1E001C01D92A135B2078D
:10028000E1F70E9427110C9424220C9400008111A4
:1002900006C0662311F082E509C081E507C0813000
:1002A00039F4662311F089EA01C08AEA0E943A0310
:1002B00081E0089581E0089581E008950C945C0147
:1002C00008950C9460011F93CF93DF9300D000D06A
:1002D0001F92CDB7DEB749835A836B833091990162
:1002E00089819A81311114C0662359F0222349F083
:1002F0000E949307182F682F89819A810E943C07DA
:1003000003C00E946707182F69817A81812F04C07A
:100310000E94930769817A810F900F900F900F9040
:100320000F90DF91CF911F910C94CE0EFC01262FE0
:10033000408151816281738184810C94630181E0E9
:100340000895CF93DF93EC0160E00E949601BE0117
:10035000DF91CF910C9461010C94FD0F0C94F90F77
:1003600008950E94E6050E94B0012FEF84E39CE00F
:10037000215080409040E1F700C000000C946B1ABF
:100380000F931F93CF93DF938C0161E00E9496013E
:10039000EC01B8010E945E01882309F444C0B80151
:1003A000CE010E94AA148823F1F1B801CE010E9467
:1003B00089188823C1F1B801CE010E94A5158823B0
:1003C00091F1B801CE010E94E517882361F1F8018F
:1003D0008281882309F1CB358DE5D807C1F050F42F
:1003E000C115FCE5DF0781F0CF3DDC45A9F40E9493
:1003F000C40C19C0CC35EDE5DE0761F0CD35DD4527
:1004000059F40E940D0C08C00E94B1010CC00E945A
:10041000160C02C00E94190CC801DF91CF911F91E8
:100420000F910C945A0180E0DF91CF911F910F91B1
:1004300008950E94A01980E00E94DF140C943702F6
:100440000E94CE130E943A020C94A61908950C94AF
:10045000260281E008950C9429020895CF93C82FB5
:100460000E9427028C2F0E942B02CF91089580E0DA
:100470000C942E020E94E5180C942E020E94E5189E
:1004800090919801891721F0809398010C942E0285
:100490000895CF93DF93CDB7DEB72B970FB6F894BF
:1004A000DEBF0FBECDBF4F83588769877A878B87A2
:1004B00061110E94590B9E012F5F3F4F86E0F901A9
:1004C00011928A95E9F785E0FE013796D9010190EE
:1004D0000D928A95E1F789819A814C815D81452B46
:1004E00031F09F3F31F491E08F3F19F403C091E068
:1004F00001C090E090FF09C049815A816B817C81E5
:100500008D819E810E947A0A05C0C9010E949F01C7
:100510008111F2CF2B960FB6F894DEBF0FBECDBF80
:10052000DF91CF910895FC01808191810E94D507D0
:100530000895CF93882309F450C0C82F8CEF8C0FF7
:10054000813AD0F46C2F80910201909103010E94B6
:100550004219882349F06C2F809102019091030188
:100560000E947A190E947B0B6C2F8091020190915E
:1005700003010E9478190CC080E28C0F883058F477
:10058000C77081E001C0880FCA95EAF70E943C0B52
:10059000CF910C947B0BEBE5EC0FE33040F4F0E0F3
:1005A000E95BFE4F808190E0CF910C940A19E8E559
:1005B000EC0FE73150F4F0E0EE0FFF1FE75EFE4F67
:1005C00080819181CF910C942019CD3E30F08C2FF9
:1005D0000E94AC11CF910C947E12CF910895882384
:1005E00089F19CEF980F913A40F4682F80910201B5
:1005F000909103010E947A190DC090E2980F9830F3
:1006000058F4877091E001C0990F8A95EAF7892F15
:100610000E94420B0C947B0B9BE5980F933020F4C7
:1006200080E090E00C940A1998E5980F973120F437
:1006300080E090E00C9420198D3E20F00E9407127B
:100640000C947E1208951F93CF93DF93182FEB0124
:100650000E949902209741F08FE99FE00197F1F7FE
:1006600000C000002197F6CF812FDF91CF911F911D
:100670000C94EF02893319F060E070E002C060E58D
:1006800070E00C942303882321F00E943C0B0C940F
:100690007B0B0895882321F00E94420B0C947B0B66
:1006A0000895CF92DF92EF92FF920F931F93CF9313
:1006B000DF937C01D62FC72FFC01128105810295A3
:1006C0000F700E94320B8823B9F01123A9F08C2FF0
:1006D000807F803421F080E28D0F883068F0809137
:1006E000380282FD09C082E00E94DB0B0E94320BBF
:1006F00091E0D82ED92601C0D12CCC2EC2948FE007
:10070000C8228C2D90E08C30910508F0CFC1FC01FF
:10071000EA5AFF4F0C94B5218C2F807FCF7088232D
:1007200011F0C295C07F112399F0CC2309F4AAC11E
:1007300080E28D0F883010F0D11104C08C2F0E9400
:100740003C0B03C08C2F0E944C0B0E947B0B9AC168
:100750008D2F0E94EF02CC2309F4A8C180E28D0FF7
:10076000883038F1DD2329F18C2F0E94520B24C0F0
:100770008C2F807FCF70803211F0C295C07FDD2337
:1007800019F0D130A1F13DC08091380282FF17C02D
:10079000112349F0CC2329F08C2F0E943C0B0E949E
:1007A0007B0B80E070C180E00E94EF02CC2309F453
:1007B0007DC18C2F0E94420B0E947B0B77C11123BD
:1007C00071F0002341F0013031F40E945C0B8C2B5E
:1007D0000E94640B6BC10E945C0B8C2B1DC000231C
:1007E00019F0013009F462C10E94710B25C0112378
:1007F00021F0063008F05AC10EC0053008F056C18D
:100800001BC0112361F0002331F0F701858180FFC7
:1008100039C18F7085838C2F0E94430347C1002309
:1008200059F0D93309F03FC1FFEF07EE13E0F15063
:1008300000401040E1F735C18C2F0E944A0336C1B9
:100840008C2F86958695837019F0813061F02EC1CA
:10085000112321F08D2F9C2F937002C080E090E037
:100860000E940A192BC1112321F08D2F9C2F937008
:1008700002C080E090E00E94201920C18D2F11233A
:1008800019F00E94AC1102C00E9407120E947E1251
:1008900015C18C2F837009F047C011110BC12D2F8A
:1008A000229526952770220F220F6D2F6F70862FAD
:1008B00090E0A0E0B0E0022E04C0880F991FAA1FAC
:1008C000BB1F0A94D2F7D4FF10C04FE050E060E0A5
:1008D00070E004C0440F551F661F771F2A95D2F79A
:1008E000409550956095709503C040E050E0BA0186
:1008F000C695C695C3708A019B01082B192B2A2B1C
:100900003B2BC901B801C23049F058F4C13019F08D
:100910000E945206CFC00E944006CCC00E946406CE
:10092000C9C00E943E06C6C0112319F08C2F8170E9
:1009300001C08695882309F4BDC02D2F22952695E8
:100940002770220F220F6D2F6F70862F90E0A0E08E
:10095000B0E0022E04C0880F991FAA1FBB1F0A9483
:10096000D2F7D4FF10C04FE050E060E070E004C068
:10097000440F551F661F771F2A95D2F74095509553
:100980006095709503C040E050E0BA01C695C695E9
:10099000C3708A019B01082B192B2A2B3B2BC90101
:1009A000B801C23049F058F4C13019F00E9417075D
:1009B00081C00E9405077EC00E9429077BC00E945B
:1009C000780678C0CF70112339F08C2F0E949E06D4
:1009D0008D2F0E9443036EC08D2F0E944A038C2FDF
:1009E0000E94BF0667C0D23F21F128F4D03F41F0FA
:1009F000D13FC1F043C0D33F19F1D43F79F03EC09D
:100A0000112341F0053008F051C08C2F8F710E94E6
:100A1000E4064CC0063008F049C0F7CF8091380298
:100A200082FF18C0112339F08C2F8F710E949E060F
:100A30003DC01123C9F38C2F8F710E94BF0636C0B1
:100A4000112329F08C2F8F710E9489062FC00E94DC
:100A500084062CC0112349F0CF718C2F0E949E0672
:100A600063E08C2F0E94C00B21C081E00E94DB0B51
:100A70000230E0F082E00E94DB0B18C0112331F05D
:100A8000002391F28D2F0E94990210C0002399F249
:100A9000D93349F41FEF27EE33E0115020403040A6
:100AA000E1F700C000008D2F0E94EF0288EF8C0D4F
:100AB000843020F40E94E5180E942E02DD20C9F047
:100AC0000E942E0B80FD15C0F70112820E94280B98
:100AD0000E949E06C7010E949A050E94280BDF9182
:100AE000CF911F910F91FF90EF90DF90CF900C94DA
:100AF000BF06DF91CF911F910F91FF90EF90DF9094
:100B0000CF9008950F931F93CF93DF93EC016881EB
:100B100079818A810E94E0078C010E943B070E9434
:100B20002C06B801CE010E945103DF91CF911F9195
:100B30000F910895CF93DF93EC01988189812B81E8
:100B40003C81232B31F08F3F31F481E09F3F19F43A
:100B500003C081E001C080E080FD1DC0CE010E9485
:100B6000C001811110C00E94320B8823A1F08A813C
:100B7000882389F08091380282FD0DC082E0DF91E8
:100B8000CF910C94DB0BCE010E948205CE01DF9148
:100B9000CF910C94A101DF91CF91089580E090E076
:100BA0000E940A1980E090E00E9420190E94590BCF
:100BB0000E947B0B0E94AF130C947E128091020165
:100BC000909103010E947C190C94CE050E94490B60
:100BD0000C94DE0592959F70963079F010F4925047
:100BE00001C09A50923068F4803F69F018F4883E52
:100BF00040F409C0843F29F406C0883E20F0813FBC
:100C000011F080E0089581E00895FC0180819181D8
:100C10000E94D5070E94EA050895CF93DF9300D084
:100C200000D01F92CDB7DEB70F900F900F900F90AE
:100C30000F90DF91CF910895CF93DF9300D000D034
:100C400000D0CDB7DEB726960FB6F894DEBF0FBE44
:100C5000CDBFDF91CF910895089508950C942D068E
:100C60000C942E060E9430066093A8017093A9018F
:100C70008093AA019093AB010C94CE050C9432069C
:100C80000F931F930091A8011091A9012091AA012F
:100C90003091AB01602B712B822B932B1F910F9105
:100CA0000C9432060F931F930091A8011091A90193
:100CB0002091AA013091AB016023712382239323F9
:100CC0001F910F910C9432060F931F930091A8016E
:100CD0001091A9012091AA013091AB0160277127E1
:100CE000822793271F910F910C9432060C942D06A6
:100CF0000E9476066093A4017093A5018093A601DB
:100D00009093A7010C94CE0560E070E0CB010C94A9
:100D100078060F931F9341E050E060E070E08A0195
:100D20009B0104C0000F111F221F331F8A95D2F7A9
:100D3000C901B8011F910F910C9478060F931F936E
:100D400041E050E060E070E004C0440F551F661FB2
:100D5000771F8A95D2F78091A4019091A501A09167
:100D6000A601B091A7018A019B01082B192B2A2B00
:100D70003B2BC901B8011F910F910C9478060F937A
:100D80001F9341E050E060E070E004C0440F551F45
:100D9000661F771F8A95D2F740955095609570959C
:100DA0008091A4019091A501A091A601B091A70105
:100DB0008A019B01082319232A233B23C901B80177
:100DC0001F910F910C9478060F931F9341E050E010
:100DD00060E070E004C0440F551F661F771F8A95BE
:100DE000D2F78091A4019091A501A091A601B091A4
:100DF000A7018A019B01082719272A273B27C90138
:100E0000B8011F910F910C9478060F931F930091D6
:100E1000A4011091A5012091A6013091A701602B9A
:100E2000712B822B932B1F910F910C9478060F93AB
:100E30001F930091A4011091A5012091A60130916A
:100E4000A70160237123822393231F910F910C9498
:100E500078060F931F930091A4011091A501209192
:100E6000A6013091A70160277127822793271F9140
:100E70000F910C9478060895292F220F920F890F55
:100E8000E82FE695E695E695877051E001C0550F8D
:100E90008A95EAF785E0E89FF0011124E656FE4FB7
:100EA00020E030E070E04081CB01022E02C0969538
:100EB00087950A94E2F7817081958427852384279A
:100EC00081932F5F3F4F2530310569F70895292F12
:100ED000220F920F890F682F669566956695982F59
:100EE000977085E0689FB001112440E050E080E0F9
:100EF000FB01E40FF51FE656FE4F208130E0092E7E
:100F000002C0369527950A94E2F721703327042E04
:100F100001C0220F0A94EAF7822B4F5F5F4F4530E2
:100F2000510531F70895BF92CF92DF92EF92FF9271
:100F30000F931F93CF93DF938C01C090A401D090A7
:100F4000A501E090A601F090A7018091A8019091E1
:100F5000A901A091AA01B091AB01C82AD92AEA2A15
:100F6000FB2ACFE1D0E0D701C6010C2E04C0B69514
:100F7000A795979587950A94D2F780FD04C021978D
:100F800090F7B12C07C0BC2EB8018C2F0E94E40E44
:100F90000197A9F38B2DDF91CF911F910F91FF90B6
:100FA000EF90DF90CF90BF900895CF93DF93EC0147
:100FB0000E949307BE010E94E40EDF91CF91089535
:100FC0001F93CF93DF93EB0190919901992321F027
:100FD000CB010E94D50713C0882349F0CB010E94A2
:100FE0009307182F682FCE010E943C0704C0CB0145
:100FF0000E946707182FBE01812F0E94E40EDF9127
:10100000CF911F9108951F93CF93DF93C091AC01AF
:1010100016E08091AD01C81799F0D0E01C9FF00157
:101020001D9FF00D1124E255FE4F408151816281D8
:101030007381848195810E941C062196C770E9CF37
:10104000DF91CF911F9108954091DE015091DF0112
:101050006091E0017091E1018091E2019091E301E2
:101060000C941C06EF92FF920F931F93CF93DF9384
:101070008091E30182958F7009F065C08091E00155
:10108000882309F460C08091AC01F090AD0110910B
:10109000DE010091DF016091E1017091E20191E0D8
:1010A0001F3F09F090E0C0910001D0910101292F6C
:1010B00096E0E92E8F1509F446C06115710521F0FF
:1010C0000F3F21F030E003C031E001C0322F90E04B
:1010D00030FD36C0E89EF001E99EF00D1124DF01DD
:1010E000A255BE4F11963C911197301329C03C91E7
:1010F000311326C012963C911297311121C01396DC
:101100004D915C911497461B570B4C175D07C0F42B
:101110008091E3018F7080618093E301ED54FE4F75
:1011200080818F70806180838EED91E00E949A05AE
:10113000DF91CF911F910F91FF90EF900C940308D6
:1011400001968770B7CFDF91CF911F910F91FF90DC
:10115000EF9008959F92AF92BF92CF92DF92EF925D
:10116000FF920F931F93CF93DF93CDB7DEB76197B5
:101170000FB6F894DEBF0FBECDBF8C0185E0F8013D
:10118000DE011D9601900D928A95E1F7D801129625
:10119000EC909091DE01E091DF012091E10130912E
:1011A000E2012115310531F0EF3F31F481E09F3F3D
:1011B00019F403C081E001C080E0B82FB1709B2E0C
:1011C00080FD47C1D8014C9111965C9111971396FF
:1011D000AD90BC9014978EEDC82E81E0D82EF09083
:1011E000E001B501621B730B2091000130910101F8
:1011F000FF2009F4D9C08091E3016217730708F05A
:1012000095C0282F207F09F052C05E1313C04913E8
:1012100011C0FE2CE1100EC08F7080618093E3013D
:101220000E942408C6010E949A058091E301F801FA
:1012300085834DC1AB2831F05F3F31F481E04F3FF2
:1012400019F403C081E001C080E080FD03C081E0AB
:101250008E2502C080E090E0F82FF170FF2E80FF15
:101260001CC08091AC012091AD0136E0821709F4D9
:101270000BC190E0389FF001399FF00D1124E25529
:10128000FE4F6181561306C06081461303C0628120
:10129000E61203C001968770E9CFFE2CEE2009F418
:1012A00016C18091E30181608093E30154C05E1315
:1012B00006C0491304C0E11002C0F80199C0C8017A
:1012C0000E940506882361F1EE2051F12091E3018F
:1012D000822F82958F7090E0029774F08091DE01EA
:1012E0009091DF0198878F831986BB86AA862C8709
:1012F000CE0107960E949A0586E0F801AEEDB1E0B6
:1013000001900D928A95E1F70E9432080E9424080C
:101310000AC05E1711F1C8010E94050681112CC098
:10132000C8010E949A05FF24F394D1C0282F207F82
:1013300081F77A2DB98AA88A6E2D89890E940D06B7
:101340008EED91E00E949A0586E0D6011D928A9565
:10135000E9F70E942408F12CBAC04913DCCFE11050
:10136000DACFF8018583C8010E949A0586E0D6018C
:101370001D928A95E9F7ABC0EE2091F22091E3012E
:10138000822F82958F7090E002970CF4B5CF8091F8
:10139000DE019091DF019A8389831B82BD82AC823A
:1013A0002E83CE010196A6CF6217730708F044C0C2
:1013B000FE2CEE2009F4B4CF5E1330C049132EC0CA
:1013C0002091E30120FD21C0822F82958F70482F4C
:1013D00050E041155105C9F0F80125834F30510502
:1013E00041F08F5F982F9295907F822F8F70892B7D
:1013F0008583C8010E949A0586E0F801AEEDB1E050
:1014000001900D928A95E1F73CC086E0F801AEEDBF
:10141000B1E001900D928A95E1F759C0C8010E9490
:101420000506811169CF8091E30181608093E3011A
:10143000C8010E949A054BC07A2DB98AA88A6E2DE0
:1014400089890E940D0686E0D6011D928A95E9F7EA
:1014500018C0EE2009F464CFC8010E940506F82EDA
:10146000882309F45DCF86E0F801AEEDB1E001908C
:101470000D928A95E1F78EED91E00E9493020E9411
:1014800032080E94240823C04D875E878D859E8583
:101490000E94D507292F22952F70223028F49F70A3
:1014A00039F0811105C00BC0243028F49F7049F435
:1014B000805E883020F0C8010E949A059F2CF92C8C
:1014C00006C0D80115969C91907F91F7F8CF8F2D8B
:1014D00061960FB6F894DEBF0FBECDBFDF91CF91FE
:1014E0001F910F91FF90EF90DF90CF90BF90AF9042
:1014F0009F9008951F93CF93DF93CDB7DEB72C97BE
:101500000FB6F894DEBF0FBECDBF4F8358876987F3
:101510007A878B879C87CE0107960E94AA0888232A
:10152000D1F09F8188852A853B85232B31F08F3F21
:1015300031F481E09F3F19F403C081E001C080E0F5
:1015400080FD47C04F81588569857A858B859C854C
:101550000E941C063EC086E0FE013796DE01119611
:1015600001900D928A95E1F7FF81E8856A857B8578
:101570006115710531F0EF3F31F481E0FF3F19F45F
:1015800003C081E001C080E080FD23C02091AD0157
:1015900030E0C9010196877099274091AC0150E075
:1015A00084179507F1F1F983EA837D836C8396E0D4
:1015B000929FD001939FB00D1124A255BE4FFE0102
:1015C000319601900D929A95E1F78093AD010E94BA
:1015D000030816E08091AC019091AD01891771F17B
:1015E000189FC001112482559E4F0E94AA0888238B
:1015F00029F1E091AC011E9FF0011124E255FE4F4C
:101600004081518162817381848195810E941C0691
:101610008091AC0190E00196877099278093AC018E
:10162000D9CF0E94E6051092AD011092AC01EEED0B
:10163000F1E086E0DF011D928A95E9F72C960FB65E
:10164000F894DEBF0FBECDBFDF91CF911F910895FB
:101650008091EC0185958595859508958091EC01A3
:10166000877008959091EC01977081E009F480E013
:1016700008958091F70108959091F701892B809347
:10168000F701089580959091F70189238093F701E0
:1016900008951092F70108959091F601892B809397
:1016A000F601089580959091F60189238093F601C3
:1016B00008951092F60108958091ED01089508951E
:1016C0000C945F0B0C94600B9091380292FD08C053
:1016D0009091ED01981721F08093ED010C94620B2D
:1016E00008958091ED01882329F01092ED0180E0AA
:1016F0000C94620B0895CF93DF93E0910201F09177
:1017000003018091F7018083E0910201F0910301D0
:1017100090818091F601892B80838091ED0188234F
:1017200081F0E0910201F09103019081892B808387
:1017300080910201909103010E94361981110E944B
:10174000710BC0910201D091030148E050E064EEBA
:1017500071E0CE010E94D521892B69F088E0FE015D
:10176000A4EEB1E001900D928A95E1F7CE01DF91F0
:10177000CF910C94F118DF91CF9108950C945F0BE9
:101780009091380292FD10C098E0899F9001112439
:10179000262B2093EC010E949E068091EC018595FA
:1017A000859585950C94BE0B0C949E061092EC01C9
:1017B00080E00C94BE0B2091EC01809582238093F5
:1017C000EC01982F977099F430E0482F082E000C08
:1017D000550B2417350759F09091380292FD07C038
:1017E0008595859585950E94BF060C94D60B089526
:1017F0009091380292FB222720F9281769F080FB8C
:1018000092F99093380280913702909138020E94A9
:10181000400C82E00C94DB0B08958091380282FB2F
:10182000882780F991E089270C94F80B81E00C94CB
:10183000F80B80E00C94F80B80E090E00E94EA2125
:1018400021E0893E9E4F09F020E0822F089582E03A
:1018500090E00C94E22183E090E00C94E221CF939D
:1018600084E090E00E94E221C82F82E290E00E9492
:10187000E2212C2F30E0A901582BCA01CF91089505
:10188000CF93C92F682F84E090E00E94F0216C2F45
:1018900082E290E0CF910C94F021AB01BC018FE08B
:1018A00090E00C940222AB01BC0183E190E00C9427
:1018B000022260E070E0CB010C94530C60E070E019
:1018C000CB010E944D0C0C94590C69EE7EEF80E028
:1018D00090E00E940E2260E082E090E00E94F02101
:1018E00060E083E090E00E94F0211092A801109245
:1018F000A9011092AA011092AB0160E084E090E08F
:101900000E94F02160E082E290E00E94F02160E01D
:1019100085E090E00E94F02160E086E090E00E9487
:10192000F0216FEF87E090E00E94F02140E050E06E
:10193000BA0188E090E00E94022260E08DE090E031
:101940000E94F02140E050E0BA0188E190E00E945E
:10195000022260E087E190E00E94F02140E050E048
:10196000BA018CE190E00E94022260E070E080E227
:1019700090E00E940E2240E050E0BA0188E190E041
:101980000E9402220C945E0C0C94650C682F8EE071
:1019900090E00C94F0210E942A1A60930302709345
:1019A000040280930502909306026093FF017093F6
:1019B0000002809301029093020208950E942A1A65
:1019C00060930302709304028093050290930602D1
:1019D0006093FB017093FC018093FD019093FE01E5
:1019E000089585B7806885BF85B7806885BF0895ED
:1019F00081E008950C94F80C08950C94FC0C0C9460
:101A0000FC0C0C94FF0C0C94FC0C0C94030D0C942B
:101A1000FC0C0E94F10C80EC9FE00E94DB180E94FD
:101A2000070D0C94050D0E94FD0C0C94FC0C0E94FB
:101A3000C30F0E942D020C9495150E94151A0E9446
:101A40008C100E94170D0E94CE130E94F6160C9463
:101A5000010D8F929F92AF92BF92CF92DF92EF9241
:101A6000FF920F931F93CF93DF93CDB7DEB72A97E3
:101A70000FB6F894DEBF0FBECDBF0E94A110982E06
:101A800081110E94CB0C88EFA82E81E0B82E00E0D7
:101A900010E0802E802F0E94E70FD82EF501C19014
:101AA0005F01C826B1F40F5F1F4F0330110589F79E
:101AB0008FEF89838A831B820E941E1A8160782F90
:101AC0009D838C8349815A816B818D810E9449025B
:101AD0002FC08091070281FD0E94ED0FE12CFF24B1
:101AE000F3948C2D8F21F1F00E94FA0C882399F049
:101AF000EE828F82DF2081E009F480E088870E94F7
:101B00001E1A8160782F9A8789874E815F81688548
:101B10008A850E944902F801E850FE4F8081F8262C
:101B2000F08206C0E394FF0CF3E0EF12DACFBBCFF4
:101B300081E0911001C080E02A960FB6F894DEBFD4
:101B40000FBECDBFDF91CF911F910F91FF90EF900E
:101B5000DF90CF90BF90AF909F908F9008950E949C
:101B6000290D0E9494150E94481781110E94DE0CD5
:101B70000E949C120C943E02CF93DF930E94E90EC8
:101B8000EC01811521E5920708F045C0811530E58B
:101B9000930708F094C0883E910528F5803E910592
:101BA00008F0F8C0883A910570F4853A910508F07C
:101BB0007CC08130910509F475C008F4E8C0049731
:101BC00008F0E8C0E4C08F3B910508F0E0C0C85AB7
:101BD000D0E0CC0FDD1FC65BDE4F0990D881C02D51
:101BE000CE019464D8C0811540E2940758F4811561
:101BF00051E0950708F0CEC08D3E910508F4C7C0AE
:101C00009065C9C0C11580E4D80708F4C0C0DF7072
:101C1000CE01906AC0C0811525E59207A8F4811510
:101C200034E5930708F095C0811543E5940708F063
:101C30007BC0811552E5950708F061C0D82FCC27ED
:101C4000CE01816F906AA7C0C11589E5D807A0F4BD
:101C5000C11528E5D20708F082C0C11536E5D307C3
:101C600008F095C08C2F0E947D0F8F7190E0D82FC7
:101C7000CC27CE0190628FC0C1154AE5D40708F485
:101C800074C0CE0190568115904208F080C08D2F0F
:101C90008F710E947D0FDD27D0628F71AE01582BAE
:101CA000CA0179C081E090E076C0C55AD0E0C8583A
:101CB000DE4F8881C82FD0E0CE0190646CC074E004
:101CC000969587957A95E1F7282F23703C2F3370EE
:101CD00081E090E002C0880F991F3A95E2F79C6876
:101CE000AC01522B9A019C2F9F709695969550E2CD
:101CF000959FE0011124C9018C2B9D2B4CC0837052
:101D0000992721E030E002C0220F331F8A95E2F7C5
:101D10009C2F9695969580E2989FE0011124C22B06
:101D2000D32BCE019C6837C08370992721E030E027
:101D300002C0220F331F8A95E2F79C2F9695969545
:101D400040E2949FE0011124C22BD32BCE019A686C
:101D500022C0D82FCC27CE01846F906A1CC0DC2F04
:101D6000CC27CE01806F906A16C08C2F8F700E9496
:101D70007D0F94E0D695C7959A95E1F7CF70D0E0A6
:101D8000DC2FCC27D0699E01282BC90104C080E03C
:101D900090E001C0CE01DF91CF910895272F30E070
:101DA000F901EE0FFF1F2E0F3F1FF90199E0899FE8
:101DB000E00DF11D1124E60FF11DEE0FFF1FE8529B
:101DC000FF4F8591949108950E94CE0E0E94BC0D04
:101DD00008958238910569F1B0F48133910509F4D1
:101DE0006DC048F48932910509F463C08A329105C7
:101DF00009F469C008958533910509F455C0893304
:101E00009105B9F00895833E910569F138F4803E5B
:101E10009105B1F0823E910509F10895863E910544
:101E2000A9F1873E9105B9F1843E910509F064C09E
:101E300023C02091370220FD4FC021FD4DC00895E1
:101E40008091370280FD44C08091380280FF44C0F9
:101E50008091370284FD42C083EE4DC080913702ED
:101E600082FF38C0F5CF8091370282FD33C0809168
:101E7000380280FD31C0ECCF8091380281FF32C042
:101E80008091370284FD2AC087EE35C080913702E9
:101E900083FF26C0F5CF8091370283FD21C080915A
:101EA000380281FD1FC0ECCF8091370285FD1CC038
:101EB0001DC08091370285FD19C016C08091370280
:101EC00086FD16C017C08091370286FD13C010C072
:101ED00089E311C082EE0FC080EE0DC080E00BC020
:101EE00086EE09C084EE07C089E205C085E303C021
:101EF0008AE201C081E390E008959091370292FF59
:101F00000DC0282F2871283019F4877F846006C0FF
:101F1000282F2471243011F48B7F886093FF0DC02B
:101F2000282F2871283119F4877E846106C0282F54
:101F30002471243111F48B7E88612091380220FFB6
:101F40000DC0382F3871383019F4877F816006C092
:101F5000382F3171313011F48E7F886021FF0DC030
:101F6000282F2871283119F4877E816106C0282F17
:101F70002171213111F48E7E886194FD877E089550
:101F800080E0089508950E941C0C811102C00E94F7
:101F9000C40C0E94270C809307020E942F0C909380
:101FA0003802809337020E94C20F0E942B0C682FC8
:101FB00070E080E090E00E943E066091A401709184
:101FC000A5018091A6019091A7010C947606E82FB7
:101FD000F0E0E45CFD4F80810895089580EA8A95E1
:101FE000F1F7089500C008950C94EE0F08950C9435
:101FF000F60F0C94F70F0C94F60F0C94FB0FF8945B
:10200000E82FE295EF70F0E031A1282F2F7081E0EA
:1020100090E001C0880F2A95EAF7982F90959323B6
:1020200091A392A1892B82A37894089584EF0E94B2
:10203000FF0F85EF0E94FF0F86EF0E94FF0F84E3E2
:102040000E94FF0F85E30E94FF0F86E30C94FF0FB1
:10205000CF92DF92EF92FF920F931F93CF93DF9374
:102060008C01C62FD0E0CE0182589E4F7C01FC012E
:1020700090819F3F09F447C0D62EF894E92FE2954E
:10208000EF70F0E081A19F7021E030E001C0220FED
:102090009A95EAF7822B81A382A12095282322A377
:1020A00078940E94F20FEBE7F1E04EE751E031E067
:1020B000C12C21912F3F89F0A22FA295AF70B0E0E3
:1020C00090968C9190E02F7002C0959587952A95F7
:1020D000E2F780FD02C0832F01C080E0C82A330FE1
:1020E0004E175F0731F7F70180818F3F11F00E9493
:1020F000FF0F61E0C11001C060E08D2D0E94F40F60
:10210000C00FD11FC882DF91CF911F910F91FF9017
:10211000EF90DF90CF9008950E94161083E0ECE3DB
:10212000F2E0DF01982F1D929A95E9F7E9E3F2E0DA
:10213000DF011D928A95E9F783E00E94E4100C9478
:10214000AC011F93CF93DF9300D01F92CDB7DEB7C2
:1021500019821A821B8260E0CE0101960E9428102B
:1021600061E0CE0101960E94281062E0CE01019646
:102170000E94281043E050E0BE016F5F7F4F89E36B
:1021800092E00E94D52111E0009709F410E0892B1C
:1021900049F089819A81AB818093390290933A0208
:1021A000A0933B02212F43E06CE372E089E392E0CD
:1021B0000E94E5100E94AE01812F0F900F900F90AA
:1021C000DF91CF911F9108950895FF920F931F9370
:1021D000CF93DF938C01F62ED72FC42F222349F003
:1021E00081E080930A020E941E1A90930902809354
:1021F000080280910A028823C1F080910802909120
:1022000009020E94361A059780F0EF2DFD2FD801A4
:102210004C2F50E0CD01801B910B841795071CF4C7
:102220008D918193F7CF10920A02DF91CF911F9188
:102230000F91FF9008950E94211C0E941D0D0C9487
:102240002D1C0E94311C0E94AF0D0C944B1C0E944F
:10225000BC190E94081C0E94090D0E941B110E94BB
:1022600021110E94130DFBCF8091110280FF06C047
:102270006091090170E0660F771F26C081FF04C0DE
:102280006091090184E005C082FF07C060910901E7
:1022900088E0689FB001112417C090911002992323
:1022A000D1F060910801961788F72091090188E024
:1022B000289F90011124929FA001939F500D1124FB
:1022C00070E0CA010E947F216038710540F46115F9
:1022D000710519F406C068E070E0862F08958FE755
:1022E000089581E008958091110280FF08C06091F7
:1022F000050170E0759567957595679521C081FF1B
:1023000006C06091050170E07595679519C082FF60
:1023100004C06091050170E010C090910F029923F4
:1023200099F0609104019617A0F780910501899FAB
:10233000C001112470E00E947F216038710540F4D3
:102340006115710519F406C061E070E0862F0895EB
:102350008FE7089581E008958D3E21F40E943411A5
:10236000819504C08E3E29F40E9434118093150299
:1023700008958F3E21F40E943411819504C0803F5E
:1023800029F40E943411809314020895893F19F4AE
:102390000E94731105C08A3F31F40E947311819528
:1023A0008093160208958B3F21F40E94731181954A
:1023B00004C08C3F29F40E94731180931702089582
:1023C0009FE0980F983078F421E030E0A90102C036
:1023D000440F551F9A95E2F7CA0190911302892B79
:1023E0008093130208958D3F21F480911102816042
:1023F0000BC08E3F21F480911102826005C08F3F97
:1024000029F48091110284608093110208958D3E19
:1024100039F49091150297FF35C01092150259C0FA
:102420008E3E29F4909115021916BCF32BC09091A1
:1024300014028F3E29F497FF25C01092140249C060
:10244000803F19F41916CCF31DC090911602893FF4
:1024500029F41916BCF4109216023BC08A3F19F4F5
:1024600097FF10C0F8CF8B3F39F49091170297FF78
:1024700009C0109217022DC08C3F21F490911702D1
:102480001916BCF39FE0980F983080F421E030E0FB
:10249000A90102C0440F551F9A95E2F7CA01809521
:1024A0009091130289238093130213C08D3F21F46E
:1024B000809111028E7F0BC08E3F21F4809111021A
:1024C0008D7F05C08F3F29F4809111028B7F80930F
:1024D000110280911402811106C0809115028111B0
:1024E00002C01092100280911602811106C08091E4
:1024F0001702811102C010920F0208950E941E1A45
:1025000020911402211104C020911502222321F0F0
:1025100090930E0280930D0220911602211104C0A7
:1025200020911702222321F090930C0280930B023A
:1025300082E192E00C94FC18EF92FF920F931F93AC
:10254000CF93DF9300D000D000D0CDB7DEB786E0C8
:10255000E2E1F2E0DE01119601900D928A95E1F739
:10256000E0901402F09015020091160210911702EB
:102570001092140210921502109216021092170275
:10258000E11003C0FF2009F45DC080910D0290911D
:102590000E020E94361AAC0190911002992339F074
:1025A00020910A0130E02417350758F04BC02091E4
:1025B0000B018AE0289F900111242417350718F099
:1025C00041C09F3F19F09F5F90931002EE2061F091
:1025D0000E9434111E1414F09FEF01C091E0989FE7
:1025E000902D112490931402FF2061F00E94341169
:1025F0001F1414F09FEF01C091E0989F902D1124BB
:1026000090931502309114023323E1F020911502CA
:102610002223C1F045EB3403C0011124992319F0A2
:102620009093140203C081E08093140235EB2303DE
:10263000C0011124992319F09093150203C081E081
:1026400080931502011103C0112309F45DC080912C
:102650000B0290910C020E94361AAC0190910F026D
:10266000992339F02091060130E02417350758F0FE
:102670004BC0209107018AE0289F90011124241764
:10268000350718F041C09F3F19F09F5F90930F02EC
:10269000002361F00E947311101614F09FEF01C027
:1026A00091E0989F902D112490931602112361F0D0
:1026B0000E947311111614F09FEF01C091E0989FD2
:1026C000902D112490931702309116023323E1F0DC
:1026D000209117022223C1F045EB3403C0011124DD
:1026E000992319F09093160203C081E0809316029B
:1026F00035EB2303C0011124992319F0909317029D
:1027000003C081E0809317028091140281110BC0F5
:1027100080911502811107C080911602811103C0BA
:102720008091170281110E947E12EB82FC820D8340
:102730001E8386E0FE013196A2E1B2E001900D9287
:102740008A95E1F726960FB6F894DEBF0FBECDBF8F
:10275000DF91CF911F910F91FF90EF900895E2E1EB
:10276000F2E086E0DF011D928A95E9F710921002EF
:1027700010920F0210921102089586E090E00C94DE
:10278000E221682F86E090E00C94F02180913F02D6
:102790008470896180933F020C94C1130E941C0CC9
:1027A000811104C00E94C40C0E94C6130E94BD1374
:1027B00080933F02282F26952695269530E02430D9
:1027C000310524F08770886180933F0280913F0239
:1027D00080FF04C086958695869501C080E00C94A4
:1027E000DF1420913F02822F869586958695482F8B
:1027F00050E04330510554F48F5F982F990F990F93
:10280000990F822F8770892B80933F0280913F021E
:10281000816080933F020E94C11380913F028695A0
:10282000869586950C94DF1480913F02982F96959B
:1028300096959695A1F0915E990F990F990F8770D3
:10284000892B80933F02887F91E009F490E080918A
:102850003F0290FB80F980933F020E94C113809158
:102860003F028695869586950C94DF1480913F02F1
:1028700080FD13C0816080933F02813019F489E0AC
:1028800080933F0280913F020E94C11380913F02DA
:102890008695869586950C94DF14089580913F0265
:1028A00080FF08C08E7F80933F020E94C11380E0AA
:1028B0000C94DF14089580913F0280FD0C944E1417
:1028C0000C94361490913F02892F869586958695B3
:1028D0008F5F8F719770843038F4880F880F880F5E
:1028E000892B80933F0202C090933F0280913F0268
:1028F000887F91E009F490E080913F0290FB80F99D
:1029000080933F020E94C11380913F028695869575
:1029100086950C94DF14843008F083E090913F0298
:102920009770282F220F220F220F922B90933F0295
:10293000987F21E009F420E090913F0220FB90F97C
:1029400090933F020C94DF140E948B1480913F02FD
:102950000C94C1139C01FB018281882349F12E3B19
:10296000FCE53F07C9F040F42C3BECE53E0769F07D
:102970002D3B3C4561F00895203C9CE5390791F0E2
:1029800070F0213C3C4589F0089583E001C080E06F
:102990000E94A41480E008950E941414FBCF0E94AA
:1029A000F113F8CF0E945B14F5CF0E946214F2CFAE
:1029B00081E00895279A2F9808952F9808958F926F
:1029C0009F92AF92BF92CF92DF92EF92FF920F93BE
:1029D0001F93CF93DF93C82F843050F4811109C027
:1029E00080918000877F809380000E94DD1406C064
:1029F000C3E080918000886080938000A091860071
:102A0000B09187002C2F30E00E94BB2123E030E002
:102A100040E050E00E9493210027122F232F342FF3
:102A2000012F122F232F332780918600909187004A
:102A30006CE070E00E946B216017710730F0C801F4
:102A400069E070E00E946B215EC0809186009091E9
:102A50008700E0908600F0908700E0918600F0917A
:102A60008700C6E0D0E0BE010E946B21060F171F51
:102A7000211D311D4801590185E0880C991CAA1CB3
:102A8000BB1C8A95D1F7C701BE010E946B216F0163
:102A9000E12CF12CA7019601260F371F411D511D76
:102AA000C501B4010E94932169017A01E091860079
:102AB000F0918700CA01B9010E945B219B01AC0122
:102AC000DF010E94CA219B01AC01C701B6010E942F
:102AD0005B21DC01CB012FE0B695A79597958795F3
:102AE0002A95D1F7009186001091870020E030E010
:102AF000081719072A073B0728F460918600709190
:102B00008700CB01BC0170938D0060938C00DF9136
:102B1000CF911F910F91FF90EF90DF90CF90BF90DA
:102B2000AF909F908F90089508950E94DA148AE0E4
:102B30008093800089E1809381008FEF9FEF9093D5
:102B40008700809386000C94CE13CF93DF93EC0123
:102B5000FB018281882309F43CC1C430FDE5DF0715
:102B600060F4CB3F9CE5D90788F49E0122503C4598
:102B70002431310508F02EC109C0C236EDE5DE076B
:102B800029F0C63AFDE5DF0709F024C10E942F0CA9
:102B90009093380280933702C1318CE5D80709F44D
:102BA000C6C008F042C0C930ECE5DE0709F49BC09E
:102BB00000F5C5308CE5D80709F485C078F4C3303A
:102BC000ECE5DE0709F478C008F07AC0C230DC45D5
:102BD00009F0F5C0809137028160EFC0C7309CE5F5
:102BE000D90709F478C008F07AC080913702806173
:102BF000E4C0CD30FCE5DF0709F487C058F4CB30E2
:102C00009CE5D90709F479C008F07BC080913702B0
:102C100088606FC0CF30FCE5DF0709F480C008F0A2
:102C200082C080913702877FC8C0CE3F9CE5D9071C
:102C300009F471C000F5C531FCE5DF0709F485C072
:102C400068F4C3319CE5D90709F475C008F095C054
:102C50000E94E605809137028F77AFC0CC3FFCE53C
:102C6000DF07A9F108F054C0CB3FDC4509F0A7C04D
:102C70008091380240C0C230EDE5DE0709F489C01A
:102C800058F4C1158DE5D80709F45AC008F069C099
:102C90008091380282602FC0C236EDE5DE0709F46C
:102CA0007CC0C63AFDE5DF0709F481C0C330DD45CD
:102CB00009F085C080E06EC08091370282607DC0DF
:102CC0008091370216C080913702886076C080916B
:102CD000380282604FC08091370280626EC080915E
:102CE000370280646AC00E94E605809137028068DE
:102CF00064C0846062C081603DC0809137028E7F75
:102D00005CC0809137028D7F58C08091370216C019
:102D10008091380218C0809138028D7F2BC080913D
:102D200037028F7E4AC0809137028F7D46C08091E6
:102D300037028F7B42C080913702877F8B7F3DC0F7
:102D4000809138028D7F8E7F15C08091370282FB83
:102D5000222720F991E0922790FB82F990FB83F9DA
:102D60002CC080913802982F909591708E7F892B7E
:102D700090FB81F98093380222C00E94E605809181
:102D8000370287FB222720F991E0922790FB87F9F1
:102D900014C081E00E94C60C12C08091370284FBEF
:102DA000222720F991E0922790FB84F906C08091B8
:102DB0003702982F909590FB80F98093370280918D
:102DC0003702909138020E94400C0E94E60580E094
:102DD00001C081E0DF91CF9108958FE891E00197E4
:102DE000F1F700C0000008950C944701CF93DF93E2
:102DF000A3E9B1E0C1E9D1E021E030E071E0A5391B
:102E0000B70759F18D91E82FE295EF70F0E041A1FD
:102E10008F70B90102C0660F771F8A95E2F7CB0168
:102E2000962F9095942391A392A1892B82A38991A7
:102E3000E82FE295EF70F0E041A18F70B90102C078
:102E4000660F771F8A95E2F7CB01962F9095942312
:102E500091A392A1892B82A3D1CF0E94ED168FB1AD
:102E6000982F9170799902C080E001C082E0892B8F
:102E700080931C0289B1982F9170499902C080E01B
:102E800001C082E0892B80931D02DF91CF910895CC
:102E90004F925F926F927F928F929F92AF92BF926A
:102EA000CF92DF92EF92FF920F931F93CF93DF9316
:102EB0000CE112E083E9C82E81E0D82E91E9E92ED9
:102EC00091E0F92E2AE1822E22E0922EC8E1D2E092
:102ED0005801512C412C34E0632E712CD501ED9119
:102EE0005D014E2F440F440FF60121916F01E22F37
:102EF000E295EF70F0E080A190E02F7002C0959510
:102F000087952A95E2F781709927D7015D917D0118
:102F1000E52FE295EF70F0E020A130E05F7002C095
:102F2000359527955A95E2F7F901E170FF2720FFC3
:102F300002C0E2E0F0E0E82BF92BE42BD801ED939E
:102F40008D01EF70F0E0EF57FE4F9081F40180812A
:102F5000890F808384304CF088818F5F888360E0A4
:102F6000852D0E94F41621E001C020E0D4018C914F
:102F70008D3F44F488818150888361E0852D0E94D3
:102F8000F41621E0F4018081082E000C990BB301A6
:102F90000E947F21D4018D934D01422A53942196A2
:102FA000B2E05B129BCF842DDF91CF911F910F91E7
:102FB000FF90EF90DF90CF90BF90AF909F908F9059
:102FC0007F906F905F904F900895CF93DF938631FD
:102FD0009C4541F5EB010E94390B982F8A81209185
:102FE000020130910301882379F09A7A81E009F493
:102FF00080E080931E02911102C069E201C065E386
:10300000C9010E9478190AC080911E02811102C074
:1030100069E201C065E3C9010E947A190E947B0B35
:1030200080E001C081E0DF91CF9108950F931F935D
:10303000CF93DF93C42FD22FFC0182818823C9F064
:10304000409321020E941E1A9093200280931F0237
:1030500080E28C0F883008F057C0C77081E001C053
:10306000880FCA95EAF7DF91CF911F910F910C94C9
:10307000430380912102481330C080911F02909138
:1030800020020E94361A883C910538F510E21D0F87
:10309000CD17B9F080E28C0F883040F4C77081E022
:1030A00001C0880FCA95EAF70E944A03183028F534
:1030B00081E09D2F977001C0880F9A95EAF70E94D2
:1030C0004303802F0E943A031830F0F4D77081E058
:1030D00001C0880FDA95EAF70AC080E28C0F8830C9
:1030E00098F4C77081E001C0880FCA95EAF7DF91B4
:1030F000CF911F910F910C944A03802FDF91CF91B4
:103100001F910F910C943A03DF91CF911F910F9172
:1031100008950F939C01CB01243F4CE5340731F116
:1031200088F4293DFCE53F07D9F02A3D4CE53407FA
:1031300079F1283D3C45A9F506E221EE41EE68ED26
:103140007CE52BC0263FFCE53F07E1F0A8F0273FD8
:103150003C4539F507E225EE46EE67EF7CE51DC0FC
:1031600007E225EE45EE69ED7CE517C006E221EEAB
:1031700040EE64EF7CE511C007E225EE44EE65EF1A
:103180007CE50BC006E221EE42EE66EF7CE505C071
:1031900008E221E045EE6AED7CE50E94161880E029
:1031A00008C0FC018281882319F01092210201C01D
:1031B00081E00F910895909397018093960108956F
:1031C00090932702809326020895E0912602F091C1
:1031D0002702309721F00190F081E02D099480E0E2
:1031E0000895E0912602F0912702309721F00280A5
:1031F000F381E02D09940895E0912602F0912702D1
:10320000309739F022E0DC012C930480F581E02D29
:103210000994089520912402309125022817390736
:1032200071F09093250280932402E0912602F091A0
:103230002702309721F00680F781E02D0994089548
:1032400020912202309123022817390771F09093C0
:10325000230280932202E0912602F0912702309708
:1032600021F00084F185E02D09940895FC01329647
:1032700097E080E0915029F021912223D9F38F5FCC
:10328000F9CF0895662349F0FC0132960896219102
:10329000621729F0E817F907D1F780E0089581E077
:1032A00008959C01FC0132969FEF80E04191461702
:1032B00089F09F3F19F4411101C0982F8F5F86302C
:1032C000A9F79F3F39F0F901E90FF11D97FDFA9534
:1032D0006283089508959C012A5F3F4FFC0142815B
:1032E000461301C01282019682179307B9F7089519
:1032F0000C9451190C946B19029626E0FC01119262
:103300002A95E9F7089508950C94831983E0809332
:1033100028020C948419811102C081E001C082E06E
:10332000809328020C9484190C948B1981E080936B
:1033300028020C9484190C94961908950C949D19E4
:103340000C949E190C949D190C949D190C949D1924
:10335000CF930E94A4190E94A1100E94A219C0E05C
:103360008C2F0E94E70F811104C0CF5FC330C1F7DB
:1033700001C081E0CF91089508951F920F920FB67A
:103380000F9211248F939F93AF93BF938091290243
:10339000811113C08091400290914102A09142029C
:1033A000B09143024196A11DB11D809340029093BC
:1033B0004102A0934202B0934302BF91AF919F910B
:1033C0008F910F900FBE0F901F901895809148021B
:1033D000843031F10E9419021092290220E488E120
:1033E00090E00FB6F894A895809360000FBE2093EC
:1033F000600083B7817F846083BF83B7816083BFB0
:103400007894889583B78E7F83BF0FB6F894A8957C
:1034100080916000886180936000109260000FBE10
:1034200008950E94E6050C94200282E084BD93E09A
:1034300095BD9AEF97BD80936E0008952FB7F894CD
:103440008091400290914102A0914202B0914302CA
:103450002FBF08952FB7F8946091400270914102F8
:1034600080914202909143022FBF08959C014FB773
:10347000F8948091400290914102A0914202B09153
:1034800043024FBF821B930B089578941F920F92B3
:103490000FB60F9211248F939F93AF93BF93809198
:1034A000400290914102A0914202B09143020196E4
:1034B000A11DB11D8093400290934102A09342024E
:1034C000B0934302BF91AF919F918F910F900FBE28
:1034D0000F901F90189581E08093E00080E2809328
:1034E000D8001092C9008FE19EE40197F1F700C067
:1034F000000087E090EBDC01809351029093520230
:10350000A0935302B09354029CE088E10FB6F89464
:10351000A895809360000FBE90936000FFCF8091CC
:1035200035020895089522E02093E9002FEF3091AD
:10353000E800215035FD06C035ED3A95F1F7000061
:103540002111F5CF2091E80025FF0BC040E050E0AD
:1035500066E070E00E94BD1C8091E8008E77809349
:10356000E8000895CF93DF9321E02093E9002FEF47
:103570003091E800215035FD06C035ED3A95F1F760
:1035800000002111F5CF2091E80025FF14C0EC01C7
:1035900040E050E068E070E00E94BD1C8091E800CF
:1035A0008E778093E80088E0FE01ADE2B2E0019002
:1035B0000D928A95E1F7DF91CF91089580932A02C9
:1035C00070932C0260932B0280914802843001F5A5
:1035D00082E08093E9008FEF9091E800815095FDA3
:1035E00006C095ED9A95F1F700008111F5CF809115
:1035F000E80085FF0DC040E050E063E070E08AE243
:1036000092E00E94BD1C8091E8008E778093E800D4
:103610000895BC0184E00C94DE1ABC0183E00C9494
:10362000DE1A80914702811109C00E944E1E0E943D
:10363000AB1E8091E20084608093E20008951092B6
:10364000470208950C949B196091440281E0611136
:1036500001C080E00C9486199091480281E094307A
:1036600009F080E0609144020C948B1942E061EC17
:1036700081E00E94C71D42E261EC82E00E94C71D0A
:103680009091480281E0943009F080E0609144021A
:103690000C94941980914A02833009F461C030F48B
:1036A000813071F0823009F49AC008958A3009F4AB
:1036B00086C08B3009F46CC0893009F0A8C020C0E6
:1036C00080914902813A09F0A2C08091E800877F89
:1036D0008093E80080914D0290914E02892B21F455
:1036E00068E08DE292E003C060E080E090E070E08E
:1036F0000E94081D8091E8008B778093E800089570
:1037000080914902813209F082C080914D029091EE
:103710004E02029708F07BC08091E800877F80937B
:10372000E8008091E80082FD05C080914802811187
:10373000F8CF6DC02091F3008091F20090E0922BC1
:10374000029731F48091F100813011F0863021F43C
:103750008091F100809335028091E8008B7753C00F
:1037600080914902813A09F052C080914D029091B6
:103770004E02892B09F04BC08091E800877F80932F
:10378000E8008091E80080FFFCCF8091180136C0EE
:10379000809149028132D9F580914D0290914E027B
:1037A000892BA9F58091E800877F8093E8000E942B
:1037B000FC1D80914B02809318010C94E6058091CA
:1037C0004902813221F58091E800877F8093E800EB
:1037D0000E94FC1D80914C028093360208958091D6
:1037E0004902813AA1F48091E800877F8093E80044
:1037F0008091E80080FFFCCF809136028093F10039
:103800008091E8008E778093E8000C94FC1D089569
:1038100084B7877F84BF0FB6F894A8958091600025
:10382000886180936000109260000FBE90E080E895
:103830000FB6F89480936100909361000FBE0C94D2
:1038400096190E944E1E0E94AB1EE2EEF0E08081AF
:103850008460808378940C9440218CE091E00C94F7
:10386000E018809148028530A9F4809148028530A3
:1038700079F40E94E619809146028823B1F30E94F0
:10388000A819882391F30E94A71C0E94E605EDCF9A
:103890000C94111A089508950C944E1C292F332767
:1038A00023303105C9F060F42130310581F0223038
:1038B000310509F044C08BE390E022E131E043C0E0
:1038C00021323105E1F02232310549F138C082E17F
:1038D00090E02DE431E037C099278130910549F01F
:1038E00028F0029761F5EAEEF0E005C0EEE0F1E0C5
:1038F00002C0E0E0F1E0849190E09F0124C06115F6
:10390000710541F061307105D1F489E090E02DE35B
:1039100031E019C089E090E024E231E014C0611583
:10392000710541F06130710551F48BE790E02FE5AE
:1039300031E009C080E490E02AED31E004C080E08D
:1039400090E020E030E0FA0131832083089580E1A7
:1039500089BD82E189BD09B400FEFDCF8091D80008
:103960008F7D8093D8008091E00082608093E0009A
:103970008091E00081FDFCCF0895CF92DF92EF921D
:10398000FF920F931F93CF93DF93EC018B017A018A
:103990000E941B1E811133C0E114F10439F0F701BC
:1039A00080819181081B190BC80FD91FC12CD12C04
:1039B0000115110519F18091E80085FD16C080916F
:1039C000E8008E778093E800E114F10449F0F701F4
:1039D00080819181C80ED91ED182C08285E00FC03E
:1039E0000E941B1E882321F30AC089918093F10055
:1039F00001501109FFEFCF1ADF0ADACF80E0DF9123
:103A0000CF911F910F91FF90EF90DF90CF9008958D
:103A100020914F02309150022617370748F0611568
:103A2000710539F42091E8002E772093E80001C059
:103A3000B901FC0120E06115710579F1809148021E
:103A40008823F1F18530F1F18091E80083FD3CC0DD
:103A50008091E80082FD2EC08091E80080FFEBCFCE
:103A60002091F3008091F20090E0922B6115710596
:103A700051F08830910538F421912093F100615084
:103A800071090196F3CF21E0089709F020E08091B9
:103A9000E8008E778093E800CECF2111CFCF0AC007
:103AA00080914802882361F0853061F08091E800C0
:103AB00083FD0AC08091E80082FFF2CF80E0089584
:103AC00082E0089583E0089581E0089520914F02F7
:103AD000309150022617370748F06115710539F407
:103AE0002091E8002E772093E80001C0B901FC0185
:103AF00020E06115710591F180914802882309F455
:103B000040C0853009F43FC08091E80083FD3DC08E
:103B10008091E80082FD2FC08091E80080FFE9CF0E
:103B20002091F3008091F20090E0922B61157105D5
:103B300059F08830910540F424912093F10031969A
:103B4000615071090196F2CF21E0089709F020E059
:103B50008091E8008E778093E800CBCF2111CCCF05
:103B60000AC080914802882361F0853061F080911D
:103B7000E80083FD0AC08091E80082FFF2CF80E078
:103B8000089582E0089583E0089581E00895982FD4
:103B9000973068F59093E900981739F07091EC0030
:103BA0002091ED005091F00003C0242F762F50E0BB
:103BB00021FD02C09F5FECCF3091EB003E7F309340
:103BC000EB003091ED003D7F3093ED003091EB0044
:103BD00031603093EB007093EC002093ED00509334
:103BE000F0002091EE0027FDE5CF80E008958F7072
:103BF0008093E90081E008958091490287FF11C018
:103C00008091E80082FD05C0809148028111F8CFC3
:103C100011C08091E8008B770BC080914802882307
:103C200049F08091E80080FFF8CF8091E8008E771E
:103C30008093E80008952091E4003091E50095E636
:103C40004091EC00842F817040FF23C08091E800F8
:103C500080FD1DC080914802882399F0853099F03D
:103C60008091EB0085FD11C04091E4005091E5008A
:103C70002417350729F3915011F09A01E1CF84E020
:103C8000089582E0089583E0089581E0089580E03A
:103C900008954091E80042FFDDCF08950E94BC1EC8
:103CA0000E94C41EE0EEF0E0808181608083E8ED38
:103CB000F0E080818F77808319BCA7EDB0E08C9114
:103CC0008E7F8C9380818F7E80831092470208952F
:103CD0000F931F93CF93DF930E94BC1E0E94C41EBC
:103CE000C8EDD0E088818F77888388818068888359
:103CF00088818F7D888319BC1092480210924402FB
:103D0000109246021092450200EE10E0F801808108
:103D10008B7F808388818160888342E060E080E0DF
:103D20000E94C71DE1EEF0E080818E7F8083E2EE8D
:103D3000F0E0808181608083808188608083F801E9
:103D400080818E7F8083888180618883DF91CF919D
:103D50001F910F910895E8EDF0E080818F7E8083C0
:103D6000E7EDF0E080818160808384E082BF81E0C4
:103D7000809347020C94681EE8EDF0E080818E7F0E
:103D800080831092E20008951092DA001092E10010
:103D900008951F920F920FB60F9211242F933F9305
:103DA0004F935F936F937F938F939F93AF93BF9343
:103DB000EF93FF938091E10082FF0BC08091E200BE
:103DC00082FF07C08091E1008B7F8093E1000E9419
:103DD0003F218091DA0080FF1FC08091D80080FFD2
:103DE0001BC08091DA008E7F8093DA008091D90029
:103DF00080FF0DC080E189BD82E189BD09B400FE6C
:103E0000FDCF81E0809348020E94111B05C019BCC0
:103E1000109248020E941F1B8091E10080FF19C090
:103E20008091E20080FF15C08091E2008E7F809338
:103E3000E2008091E20080618093E2008091D800EE
:103E400080628093D80019BC85E0809348020E946C
:103E5000241B8091E10084FF30C08091E20084FF48
:103E60002CC080E189BD82E189BD09B400FEFDCF8F
:103E70008091D8008F7D8093D8008091E1008F7E63
:103E80008093E1008091E2008F7E8093E200809138
:103E9000E20081608093E20080914402882311F067
:103EA00084E007C08091E30087FD02C081E001C08B
:103EB00083E0809348020E942C1B8091E10083FFE5
:103EC00029C08091E20083FF25C08091E100877FB7
:103ED0008093E10082E08093480210924402809136
:103EE000E1008E7F8093E1008091E2008E7F8093DD
:103EF000E2008091E20080618093E20042E060E0B5
:103F000080E00E94C71D8091F00088608093F000DF
:103F10000E94221BFF91EF91BF91AF919F918F91D2
:103F20007F916F915F914F913F912F910F900FBEB5
:103F30000F901F9018951F920F920FB60F92112499
:103F40002F933F934F935F936F937F938F939F93A1
:103F5000AF93BF93CF93DF93EF93FF93C091E900AB
:103F6000CF708091EC00D82FD17080FDD0E81092F6
:103F7000E9008091F000877F8093F00078940E94A0
:103F8000DF1F1092E9008091F00088608093F000BC
:103F9000CD2BCF70C093E900FF91EF91DF91CF91CE
:103FA000BF91AF919F918F917F916F915F914F9151
:103FB0003F912F910F900FBE0F901F9018951F9358
:103FC000CF93DF93CDB7DEB7AA970FB6F894DEBFD5
:103FD0000FBECDBFE9E4F2E08091F100819322E0D1
:103FE000E135F207C9F70E944A1B8091E80083FF80
:103FF0002EC18091490290914A02492F50E04A30E7
:10400000510508F024C1FA01EE59FF4F0C94B52177
:10401000803821F0823809F01AC108C08091450229
:1040200090914602992389F082600FC080914D02E1
:104030008F70873008F00BC18093E9008091EB000E
:1040400085FB882780F91092E9009091E800977F1E
:104050009093E8008093F1001092F100D1C0282FD6
:104060002D7F09F0F4C0882319F0823061F0EFC091
:1040700080914B02813009F0EAC0933009F080E072
:10408000809346022EC080914B0281112AC08091FC
:104090004D028F702FEF280F263008F0D8C0809384
:1040A000E9002091EB0020FF1CC0933021F48091A7
:1040B000EB00806214C09091EB0090619093EB0054
:1040C00021E030E0A90102C0440F551F8A95E2F7B4
:1040D0004093EA001092EA008091EB0088608093A0
:1040E000EB001092E9008091E800877F8093E80060
:1040F0000E94FC1DACC08111AAC010914B021F7719
:104100008091E3008078812B8093E3008091E80028
:10411000877F8093E8000E94FC1D8091E80080FF6B
:10412000FCCF8091E30080688093E300111102C00E
:1041300082E001C083E08093480289C080588230C9
:1041400008F085C080914B0290914C028C3D53E069
:10415000950779F583E08A838AE289834FB7F894DB
:10416000DE01139620E03EE051E2E32FF0E05093B1
:104170005700E49120FF03C0E295EF703F5FEF70BE
:104180008E2F90E0EA3010F0C79601C0C0968D9354
:104190009D932F5F243149F74FBF8091E800877FBF
:1041A0008093E8006AE270E0CE0101960E94081D4B
:1041B00016C060914D0270914E02AE014F5F5F4F8D
:1041C0000E944C1CBC01892B09F441C09091E8006D
:1041D000977F9093E80089819A810E94661D809163
:1041E000E8008B778093E80032C0803881F58091B9
:1041F000E800877F8093E800809144028093F1007B
:104200008091E8008E7772CF811121C080914B029E
:1042100090914C0299270297D4F48091E800877F0F
:104220008093E80080914B02809344020E94FC1D21
:1042300080914402811106C08091E30087FD02C095
:1042400081E001C084E0809348020E94361B809187
:10425000E80083FF0AC08091E800877F8093E80030
:104260008091EB0080628093EB00AA960FB6F894E1
:10427000DEBF0FBECDBFDF91CF911F91089508958E
:10428000CF93809148028823A1F0C091E900CF70BC
:104290009091EC00892F817090FD80E8C82B1092DE
:1042A000E9008091E80083FD0E94DF1FCF70C0937A
:1042B000E900CF910895DB018F939F930E94CA215B
:1042C000BF91AF91A29F800D911DA39F900DB29FB2
:1042D000900D11240895AA1BBB1B51E107C0AA1F12
:1042E000BB1FA617B70710F0A61BB70B881F991F97
:1042F0005A95A9F780959095BC01CD01089597FB3B
:10430000072E16F4009407D077FD09D00E946B2188
:1043100007FC05D03EF4909581959F4F08957095C8
:1043200061957F4F0895A1E21A2EAA1BBB1BFD01C8
:104330000DC0AA1FBB1FEE1FFF1FA217B307E40784
:10434000F50720F0A21BB30BE40BF50B661F771FDC
:10435000881F991F1A9469F76095709580959095BC
:104360009B01AC01BD01CF010895EE0FFF1F059029
:10437000F491E02D0994A29FB001B39FC001A39FC7
:10438000700D811D1124911DB29F700D811D11248E
:10439000911D08950E94BB21A59F900DB49F900D83
:1043A000A49F800D911D11240895FB01DC0104C020
:1043B0008D910190801921F441505040C8F7881B1D
:1043C000990B0895F999FECF92BD81BDF89A99276E
:1043D00080B50895A8E1B0E042E050E00C941622C8
:1043E000262FF999FECF92BD81BDF89A019700B4AE
:1043F000021639F01FBA20BD0FB6F894FA9AF99A4E
:104400000FBE08950396272F0E94F1210E94F021EC
:10441000252F0E94F121242F0C94F1210196272FA2
:104420000E94F1210C94F021DC01CB01FC01F999EF
:10443000FECF06C0F2BDE1BDF89A319600B40D92F0
:0C44400041505040B8F70895F894FFCFA9
:10444C00C800EE01280850011E0A14018F1AB21A76
:10445C00931A0D1B091B921A01E200E900EA00B540
:10446C0000B600B700CD008301CC008A0192019404
:10447C00012102230224022502260227022A02B36A
:10448C0000B4006F007000818283E200E900EA0052
:10449C00B500B600B700CD008301CC008A019201B3
:1044AC0094012102230224022502260227022A0259
:1044BC00B300B4006F007000818283343536F4F59C
:1044CC00F600FF0100010000FFFF0000010001FFEA
:0644DC0000F191F09000D8
:00000001FF
